:03000000020003F8
:1000030075812378237600D8FC900000AE83AF82FD
:100013009000001200416005E4F0A380F690009F79
:1000230012004A9000A312004A9000A712006890A1
:1000330000AD12006875D0001200D20200B3EF6564
:10004300827003EE658322E493F8740193F97402DA
:1000530093FE740393F5828E83E869700122E4931F
:10006300F6A30880F4E493FC740193FD740293FEF9
:10007300740393FF740493F8740593F582888312D1
:100083000041700122E493A3A883A9828C838D820B
:10009300F0A3AC83AD828883898280E3242400B5F6
:1000A300242400B5000000B500B5000000B500B57C
:0200B30080FECD
:1000B500E4F520F521C3E5219498E520648094BA00
:1000C500500A0521E5217002052080E922C280C27F
:1000D500901200B5C280D2901200B5D280D2901293
:0B00E50000B5D280C2901200B580E28E
:00000001FF
